S12300000F8E01FFCE10006F351C3C201D3C408622A709CE1000BD01101D0040BD0145BD8B
S123002001451C00408601B7500286AAB750178655B750188612B750198640B7500086FF38
S1230040B750AFB7509F4FB750EFB75000BD018ACE10006F2CCC300CA72BE72DCE1000BDAA
S1230060014EC17726352622BD0107171F2E20FCE62F18E70018E6001F2E80FCE72F1808FC
S12300804A26E9C6EEBD016A20D2C141260D8D77BD011C18E600BD016A20C1C15226228D33
S12300A06617188C5000250E188C6000240818E600F65004200318E600BD016A18084A2647
S12300C0E1C16627037E005C8D3386AAB7D5558655B7AAAA86A0B7D5558640CE6000E60078
S12300E018E7000818084A26F5BD0145BD0145BD0145CE1000C6AABD016A7E005CBD014E0B
S123010017BD014E188F398DF47E014E1F0820041D0820391C0820398606201518E1002763
S1230120238616188C103F26048DE586068D028602A73B18E7006C3B3CCE0D050926FD38C2
S12301406A3B6F3B393CCE0D050926FD3839183C18CE2710CE100018092607BD010C18CE0D
S123016027101F2E20EE1838E62F1F2E80FCE72F3986FF97074F9703860ACE0D050926FDC4
S12301804A26F79603888020ED398638B74000BD01458638B74000BD01458638B74000BD2B
S12301A00145860CB74000BD01458601B74000BD01458606B74000BD01458654B74001BDD3
S12201C001458665B74001BD01458673B74001BD01458674B74001BD01453900010203C8
S9030000FC
